:1000000012C02BC02AC029C028C027C026C025C0C6
:1000100024C023C022C021C020C01FC01EC01DC0DC
:100020001CC01BC01AC011241FBECFE5D4E0DEBF28
:10003000CDBF10E0A0E6B0E0E0E9F0E002C005903E
:100040000D92A036B107D9F710E0A0E6B0E001C0EC
:100050001D92A036B107E1F70DC0D2CF9C0106C0BA
:1000600080EF90E00197F1F72150304021153105E4
:10007000B9F70895CFE5D4E0DEBFCDBFA59AAD981E
:1000800084EF91E0EBDFAD9A84EF91E0E7DFF7CF0B
:00000001FF
